:1010BF00323235730032393220410000480050A0DF
:1010CF00323932204200004900C8A0323932204361
:1010DF0000004A0140A0323932204400004B01B8D1
:1010EF00A032323700000000230230A03238312006
:1010FF00413100380302A0323831204231003A0327
:10110F006BA0323831204331003C03D4A032383148
:10111F00204431003E043DA03238312041320039A5
:10112F0004A6A0323831204232003B050FA03238DE
:10113F0031204332003D0578A0323831204432004F
:10114F003F05E1A03231300000000020064AA032F6
:10115F00363620410000320AFAA0323636204200DD
:10116F0000330B63A032363020410000300BCCA08F
:10117F0032363020420000310C62A0323539204126
:10118F000000280CF8A032353920420000290EC982
:10119F00A0323539204300002A109AA03235392069
:1011AF004400002B126BA0323235000000002114D6
:1011BF003CA032323573000000221856A03239316C
:1011CF0020410000441973A03239312042000045FC
:1011DF0021F2A032343920410000242A71A0323587
:1011EF003020420000423B9FA032393620410000A0
:1011FF00544C09A032353620413100345249A032C7
:10120F00353620413200365393A0323536204231E5
:10121F00003554DDA032353620423200375627A034
:10122F00323732000000005E5771A0323631204154
:10123F0000002C6905A0323631204200002D6AD6FD
:10124F00A0323631204300002E6CA7A03236312059
:10125F004400002F6E78A0323835462041004C00F4
:10126F0050A2323835462042004D00BCA2323835EC
:10127F00422041004E0128A2323835422042004F11
:10128F0001DCA232303600000000500290A2323052
:10129F0037000000005303DAA23234392042000035
:1012AF00250524A232323200000000401000A23285
:1012BF003936204200005534B8A232333020410075
:1012CF0000563AF8A232333020420000573BE8A2D2
:1012DF0032333020430000583CD8A2323330204400
:1012EF000000593DC8A2323530204300005140E87C
:1012FF00A232353020440000525152A232353020F4
:10130F004100004161BCA2323233204D00005A101F
:10131F0000A2323233204100005B7226A2323531F7
:10132F00204100005C0000A3323531204200005DF7
:03133F004000A3C8
:102C9A0090030FE0FCA3E0FDA3E0FEA3E0FFE4FA4B
:102CAA00F9F8EF2401FFEA3EFEE93DFDE83CFC901D
:102CBA00030F0209117D017C0090030FE0F8A3E0E5
:102CCA00F9A3E0FAA3E0FBC30208B5900299A3E0D6
:102CDA00FAA3E0F5828A8322A3E0FAA3E0F90209C3
:012CEA00EFFA
:091A1B00E4F5B1F5A975B28322CE
:1036FC0075A407E4F5A5F5A675A71C75D40F75E19F
:05370C000475E2C22279
:0E386A00E4F592759330F594F595759104226E
:1031E700E4FFFEE4FCFD0DBD00010CBC13F8BD8837
:1031F700F5E5C130E505E4FEFF80050FBF00010ED0
:09320700D3EF94F4EE940140DAD7
:01321000229B
:1017BE00E490030BF0A3F0A3F0A3F0F5D9121A1BDB
:0C17CE001236FC12386A1233C212359138
:1017DA0090030F12091D000000007FF87E24122CCE
:0817EA00BF5005122C9A80F299
:1017F20012375012304212378C12392F1238E090C1
:1018020003B3E0FF12353A1238EC1233C2D2AF43BF
:0C181200E6811231E7E490030DF0A3F032
:10181E0090030F12091D000000007F807E38122CED
:08182E00BF5005122C9A80F254
:1018360012391912390390030EE004F07006900372
:101846000DE004F0C390030EE0940490030DE064F1
:0518560080948040C3F6
:10185B0090030F12091D000000007F007E717D02B6
:0A186B00122CC15005122C9A80F0D7
:101875001236D090030BE07002A3E0603C90030C9D
:10188500E024FFF090030BE034FFF0E07002A3E0EA
:10189500701453E6EF7BFF7A1079BF7D1AFC122C8A
:1018A5004343E6108013301310E490030BF0A3F0CC
:1018B50090029C122CE21238EC1233E7EF6073535E
:1018C500E6EF122DD4EF1209C9191401190F0219E7
:1018D500000418FB08191C0919230A18ED1019052D
:1018E50020190A400000192BC21390030B74FDF058
:1018F500A374E8F0803090030380179002FE8012F5
:101905009002D5800D9002D28008900295800390B8
:1019150002EA122CE2800F122CD57F018005122CD1
:10192500D57FFF1209F343E6101233E7EF709012EB
:1019350038EC1230DAEF70030218789003C0E02417
:10194500F6601524FE603A240A60030218787D01CA
:101955007FFE1238F80218789003C1E0FF12349820
:1019650090030AEFF0E075F00BA424C4F974103568
:10197500F0FA7BFF9003C2E0FD7C00122C430218B5
:0A198500781239191239030218789C
:031A2D0002323B47
:10323B00C0E0C083C0829003C4E004F0E05407F008
:10324B00700D900208E030E004B2838002D2835309
:09325B00913FD082D083D0E03213
:10349800E4FE75F00BEEA424CBF582E5F03410F5CC
:1034A80083E493B50703AF06220EEEB43AE47FFF38
:0134B80022F1
:10381D000001FF00FF000001010000FF00FF01009B
:0836130041020600410207001C
:10362B0053E6EFE518851983851A8222900366E02D
:08363B00FBA3E0FAA3E0F92271
:0529E500900365EFF016
:1029EA00E5172401FFE43516FAA907A37401F0A339
:1029FA00EAF0A3E9F012363774019002896B700885
:102A0A00E965827003EA6583700D90036604F0A39A
:102A1A007402F0A37409F012363712362E6B70085E
:102A2A00E965827003EA6583601E900365E0851795
:102A3A0082851683F0900366A3E0FAA3E0AE028EC5
:082A4A0016F517900365E0F09A
:012A52002261
:102DD40012362B6401700AE51765827004E51665E6
:102DE400837003FF802FAB18051AE51AAA19700225
:102DF400051914F912079DFF74019002896B700A7A
:102E0400E51A65827004E519658370097518017502
:082E14001902751A0943E610CA
:012E1C002293
:1033E70012362B6401700AE51765827004E51665CD
:1033F700837003FF800AAB18AA19A91A12079DFF49
:0334070043E61089
:01340A00229F
:031A240002206C31
:10206C00C0E0C083C082C0D075D000C001C002C027
:07207C0003C005C006C00708
:0620830020DF03022146EC
:10208900E5B030E00F900206E0700E04F07F2012F8
:1020990029E58005900206E4F0E5B030E10F9002F1
:1020A90007E0700E04F07F401229E58005900207D1
:1020B900E4F0E590541FF514651E6019E59030E4CD
:1020C90002D213E514651E900362F0541F60037574
:1020D9001C0385141EE51C6062151CE51C705CE57B
:1020E9001D6514900362F030E00AE51420E0057FD5
:1020F900011229E5900362E030E10AE51420E105C7
:102109007F021229E5900362E030E20AE51420E239
:10211900057F041229E5900362E030E30AE5142003
:10212900E3057F081229E5900362E030E40AE5142B
:0D21390020E4057F101229E585141DC2DF8A
:0621460020D80330D95D32
:10214C00900362E580F0C2D9C2D8E0FF651B54C091
:10215C00604BEFC4131354037E005403FFE51BC400
:10216C00540CFDED4F241DF582EE3438F583E493C9
:10217C00FF900363F0A3E515F0EF2515F515E06569
:10218C001530E113200F10900363E0B401047F09B4
:0D219C0080027F0A1229E5900362E0F51B26
:1021A900D007D006D005D003D002D001D0D0D0823C
:0521B900D083D0E032EC
:0F383D0043E60875DA3175DB3175D983D2DE22A7
:1035910012383D7B017A0279098B188A19891A8AB6
:0B35A100168917E4900208F002316563
:10316500900208E0FF30E004C2838002D283EF3092
:10317500E104C2958002D295EF30E204C296800246
:0C318500D296EF30E303C29722D29722CB
:0B38F800900208E05FF04DF002316527
:1034FB00E475F00112086785F082F58322A3F09042
:10350B00FFFE0209F575B7A575B7F18F828E832281
:1035E100A2AFE433FDC2AF758F03123510E4F0F5DD
:0835F1008FAF05EF24FF92AF3C
:0135F90022AF
:1035C700A2AFE433FCC2AF758F01123510EDF0E402
:0935D700F58FAF04EF24FF92AF61
:0135E00022C8
:102D8800900333EEF0A3EFF0A3ECF0A3EDF0EB4AE1
:102D98006039900333E0FEA3E0FFA3E0FCA3E0F575
:102DA800828C83E0FD1235C7EB1B70011A90033645
:102DB800E004F07006900335E004F0900334E0047A
:0C2DC800F070CB900333E004F080C322D5
:081A1000E4900004F0A3F022B1
:10332A00900004E0FEA3E0FF1235E1900004E0FE05
:10333A00A3E0FF7C007D067B007A02122D88E490D0
:06334A000004F0A3F022D4
:0A28FB00A905900331EEF0A3EFF001
:10290500EE54FEFE900004E0FCA3E0FD7002EE6CC8
:102915006045ED4C600312332A900331E0FEEE541E
:10292500FEFE7F00900004F0A3EFF0900000EEF0B3
:10293500A3EFF0A37400F0A37406F07E02900000EC
:102945001234FBE493FD9000021234FBEDF0EF1F0F
:1029550070011EEF4E70E6900331E0FCA3E0FDEC44
:0F2965005401FC74062DF58274003CF583E9F0F3
:012974002240
:102D3B0012350AEAF0EB123508ECF0ED123508EE1D
:102D4B00F0A3EFF0900004120A1974FFF5F01208CB
:102D5B006745F06022852883852982E475F001128E
:102D6B000867AFF0FE852883852982A3A31234FB65
:0D2D7B00E0FD1228FB80CD9000060209F556
:1021BE00008040C020A060E0109050D030B070F091
:1021CE00088848C828A868E8189858D838B878F801
:1021DE00048444C424A464E4149454D434B474F431
:1021EE000C8C4CCC2CAC6CEC1C9C5CDC3CBC7CFCA1
:1021FE00028242C222A262E2129252D232B272F231
:10220E000A8A4ACA2AAA6AEA1A9A5ADA3ABA7AFAA0
:10221E00068646C626A666E6169656D636B676F6D0
:10222E000E8E4ECE2EAE6EEE1E9E5EDE3EBE7EFE40
:10223E00018141C121A161E1119151D131B171F100
:10224E00098949C929A969E9199959D939B979F970
:10225E00058545C525A565E5159555D535B575F5A0
:10226E000D8D4DCD2DAD6DED1D9D5DDD3DBD7DFD10
:10227E00038343C323A363E3139353D333B373F3A0
:10228E000B8B4BCB2BAB6BEB1B9B5BDB3BBB7BFB10
:10229E00078747C727A767E7179757D737B777F740
:1022AE000F8F4FCF2FAF6FEF1F9F5FDF3FBF7FFFB0
:09393900E0FBA3E0FAA3E0F9228F
:01396500223F
:10353A00EF30E004D2808002C280EF30E104D28111
:0E354A008002C281EF30E203D28222C28222CE
:103750007F381237647F061237647D0EE4FF12381B
:04376000BC02396509
:10376400900340EFF0123643EF20E7F9900340E076
:04377400FF022FA081
:1036430075A0FFC2B3D2B4D2B27F14DFFEAFA0EF36
:073653009021BE93FFC2B2FB
:01365A00224D
:053960007F0102376445
:102FA000EF9021BE93F5A07FC87E00EF1F70011E39
:102FB000EF4E70F7C2B3C2B4D2B27E007FC8EF1F2B
:102FC00070011EEF4E70F7C2B27E007FC8EF1F7017
:062FD000011EEF4E70F738
:012FD60022D8
:102FD700EF3395E0FE74BE2FF58274213EF583E44E
:102FE70093F5A0C2B4D2B2D2B37FC87E00EF1F70F0
:102FF700011EEF4E70F7C2B27E007FC8EF1F70014F
:053007001EEF4E70F702
:01300C0022A1
:0C38BC009003C5E05FF04DFFF0023764A0
:0E387800AE07123643EF20E7F9AF06022FD756
:10310A00900340EBF0A3EAF0A3E9F09003401239F0
:10311A003912079D6017900340A3E475F001120865
:0E312A0067A9F0FA12079DFF12387880DE22A6
:1031380090033AEBF0A3EAF0A3E9F0123960E4FD5A
:10314800FF1238C890033A12393912310AE4FD7F68
:0D315800011238C890033D12393902310AC6
:0C38C800EF75F040A42D2480FF0237644F
:05326400900317EDF0DE
:10326900AF01AB0790031874FF1208DEEC4D4E4F07
:103279006010900317E08B828A83F00BBB00010A70
:0232890080E2E1
:01328B002220
:10368B00E4FD0FEFAA0670010E14F5828A83E06049
:06369B00030D80EEAF05F7
:0136A1002206
:0734B900EFF0A90512384CE9
:1034C000E50BB50FFBE50AB50EF6E50BB513F1E517
:0A34D0000AB512EC20C5E97F0122C5
:0630DA00121A27EF602727
:1030E00090032F7403F0A374BFF012321190032FDA
:1030F000E475F00112086785F082F583EFF012396C
:0731000054EF70E67F01228D
:033107007F002224
:0E384C00E4FFFE0FBF00010EBE05F8BFDDF564
:01385A00224B
:10371100AB0712384C1234C0E4FF12198FAF0312F9
:05372100198F0238D4ED
:10372600AB0712384C1234C07F0112198FAF031247
:05373600198F0238D4D8
:0B3903001234C07F1412198F0238D458
:0B390E001234C07F1512198F0238D44C
:0B3919001234C07F0B12198F0238D44B
:10328C0090032F1234B97F2D12198F90032FE0FF6A
:10329C0012198FAF0112198FAF0312198F900332CD
:0832AC00E0FF12198F0238D473
:1032B40090032F1234B97F2E12198F90032FE0FF41
:1032C40012198FAF0112198FAF0312198F900332A5
:0832D400E0FF12198F0238D44B
:10319100A907AE057F3112198FAF0112198FAF0642
:1031A10012198FAF0312198F900329E0FF12198FA3
:0B31B10090032AE0FF12198F0238D4AF
:1031BC00A907AE057F3212198FAF0112198FAF0616
:1031CC0012198FAF0312198F90032AE0FF12198F77
:0B31DC0090032BE0FF12198F0238D483
:102EAC00202020202020446F6E6520202020200030
:102EBC002000437264204E6F7420466F726D6174F3
:102ECC00746400466F7220507265736574730020D1
:102EDC00202020496E76616C69642020202020001F
:012EEC00FFE6
:07361B004403A000000000C1
:101BDC00903A7975F00DED12094EEC75F00DA425C7
:101BEC0083AF82900324F0A3EFF090031EE09003E8
:101BFC002175F00DA42479F9743A35F0FA74FFF0DC
:101C0C00A3EAF0A3E9F02212094EEE75F00BA4251D
:101C1C0083F583E493FE740193FDEEFB90031FE0C8
:101C2C00FEA3E09010CE75F00B12094EEE75F00B82
:101C3C00A42583F583E49322A37C007D0B1207EA91
:101C4C0074C42FF974103EFA7BFF22900321A3E495
:101C5C0075F001120867FEAFF0900324E475F001F3
:101C6C0002086790039178927C03E075F00DA42430
:101C7C0079F9743A35F0FA7BFF7D017E007F0D22F5
:101C8C0090033274FFF0A3742EF0A374BCF07BFFAE
:101C9C0022900318E0FF9003C1E0227BFF7A3A798F
:101CAC0075900336E4F0A37402F07D8A7C012290D7
:101CBC00031DE0FCA3E0FFECFD9011CBE493FB22B1
:101CCC00E024FFFFE434FFFE90031FE0FCA3E0FDE3
:101CDC0022FF900336E06EF0A3E06FF022E0F8A351
:101CEC00E0F9A3E0FAA3E0FBD30208CBC3900320F6
:101CFC00E0940D90031FE06480948022E0FEA3E04A
:101D0C00FFC3943AEE648094802224FFFEE434FFF7
:101D1C0090031FF0A3CEF022A42479F582E5F034D1
:101D2C003AAF82FE2290031AE0FF900318E022E4FF
:101D3C0090031FF0A3F022E0FBA3E0FAA3E0F9026A
:101D4C00079D900320E004F02290031FE004F02292
:0A1D5C009FEE6480F8EC648098228A
:10342F0012332A121CA712287E90032FEEF0A3EF5F
:10343F00F07A007B027C037D2F7E3A7F73122D3B47
:03344F0002332A1B
:10365B00121A107A007B047C037DB17E3A7F7512BF
:08366B002D3B12342FC2112285
:102CEB00E49003B1F0A3F0A3F0A3740FF012365BE2
:102CFB00121A107B017A03799290031812091D00A6
:102D0B0000000DE4FD123264900313740DF0E4F532
:102D1B001F7A007B0D7C037D9275F00DE51F121D54
:102D2B0024122D3B051FE51FC3941E40E402342FD4
:10304200121CA712287E903A737401936F7003E4E6
:10305200936E6003122CEB78B17C037D017BFF7AC7
:103062003A79757E007F04120777E490039FF0900F
:043072000391F022B4
:10378C00121C6F12077790039F78A47C03121C768F
:03379C00020777AA
:0730A900900318EB121C0B51
:1030B000A3743AF0A37479F0121A10900318A3E0E5
:1030C000FAA3E0AC02FD90039FE075F00D121D2401
:0A30D0007A007B0D122D3B02342F15
:093942007B017A0379A40230A98B
:10379F00301209121C6F12077712394230110312BF
:0337AF00365B2264
:1036D00090039FE0FF900391F012371112378CE4B2
:0636E000FD7FFE0238F838
:1035AC007B017A0379921230A912378C90039FE039
:0B35BC00FF123726E4FD7FFE0238F806
:0D287E00900331EB121C0BA3ECF0A3EDF066
:10288B0090033474FFF5F012086745F0605990031C
:10289B0031E0FBA3121C68A9F0FA12079DFD3395DA
:1028AB00E0FC900336E0FFEF6DFDA3E0F8E4F0E809
:1028BB00900336F0ECC4F854F0C868FEEDC4540F26
:1028CB0048FFEE6CFEEF6DFF121CE1EF7805C33392
:1028DB00CE33CED8F9121CDDEF7807C333CE33CE0F
:0F28EB00D8F9121CDD8099900336E0FEA3E0FFC0
:0128FA0022BB
:100E1100E490031AF090031CF0A2AF33900323F087
:100E210012256F4003021094121D3B90031F121DE7
:100E3100084003020F3E9010CB75F00BEF121C35EA
:100E4100900318F064227003020F3390031F121CE9
:100E5100447F011226BE90031FE0FEA3E09010CC58
:100E610075F00B300011121C13900332F09003182F
:100E7100E0FF1232B4800F121C13900332F0900382
:100E810018E0FF12328CC20190032912091D0000E3
:100E91000006E4900319F0900319E0FFE4FCFDFE65
:100EA100900329121CE940241230DAEF60119003FB
:100EB100C0E0B4300A121C9DB50704D201800D7F39
:100EC10001123475900319E004F080CB3001639076
:100ED100031FE0FEA3E0FF7C007D0B300007121C26
:100EE100497F038005121C497F021226BE7F011231
:100EF10034759003A0E0FCA3E0FDA3E0FEA3E02491
:100F010001FFE43EFEE43DFDE43CFC9003A0120938
:100F110011E4FFFE7D40FC9003A0121CE950131266
:100F210030DAEF60CD9003C0E0B42FC6121C9DB53E
:100F310007C0121D4E7003121D55020E2C90039115
:100F4100E0900328F09011C9E493FF74019390039A
:100F51001DCFF0A3EFF0C2AF43C15E200003020F2B
:100F6100EA7F031210AC121A10900321E0FEA3E0F5
:100F7100FF7C007D0D1207EA74792FF9743A3EFA6D
:100F8100900324121C09121D3B121CBBE490033F69
:100F9100F0D20312248D90031BEFF0FD900324A3E4
:100FA100121C68FEAFF01228FB90031EE004F070E3
:100FB1000690031DE004F0121D4E7003121D551220
:100FC1001CF840C512342F900322E004F070069003
:100FD1000321E004F0C3900322E0941E900321E07A
:100FE1006480948040800210747F021210AC9003E0
:100FF10021E0FEA3E0FFC3941EEE64809480507351
:10100100903A7975F00DEF12094EEE75F00DA425A9
:1010110083AF8290032DF0A3EFF0121D3B90032DBF
:10102100E0FEA3E0F5828E83E493900327F0121C87
:10103100BB90032D121C6885F082F583E493900325
:101041003FF0C20312248D90031EE004F07006905D
:10105100031DE004F0121D4E7003121D55121CF801
:1010610040BB900322E004F07006900321E004F0FD
:10107100020FEF1233C2900323E024FF92AF121C40
:101081008C7A2E79AC122EED900328E0900391F02A
:1010910002378C90033274FFF0A3742EF0A374CF47
:0A10A100F07BFF7A2E79BE122EEDCF
:1010AB00227BFF7A1179C11226BE900321E4F0A3B3
:0410BB00740FF0229C
:0F1A3000900319EDF0900318EFF090031AEBF00C
:101A3F00B5070E900319E0FF90031BE0B507028076
:101A4F001F121D31C39F5009A3E0FEEF9E5002806D
:101A5F000F121D31FED39F401190031BE09E400AD1
:101A6F00121C8C7A2E79DB021BC2E490031CF090BF
:101A7F00031CE0FFC3943A4003021B1575F00BEFF4
:101A8F00A424CBF582E5F03410F583E49390031D85
:101A9F00F0642260687F01121BC690031D121D3473
:101AAF00FDA3E0FBA3E090032AF090031BE090035B
:101ABF002BF01231BCE490031EF01230DAEF602CE1
:101ACF009003C0E06430702490031D121CA06F704F
:101ADF001B7F05121BC61230DAEF60FA9003C0E0CD
:101AEF00B42FF390031D121CA0B507EA7F01123427
:101AFF007590031EE004F0E0C3940540BD90031CF5
:101B0F00E004F0021A7E7BFF7A1179C17F0512265D
:101B1F00BE900318E01490031CF090031AE0149089
:101B2F00031EF0900319E014FF90031CE0FED39FF7
:101B3F005077EE900324121BFD90031EE075F00DFD
:101B4F00A42479F9743A35F0FA900321121C09E4B0
:101B5F0090031FF0900321121D43900320F0AE025B
:101B6F00AF01900324121D43FD1228FB12342F9056
:101B7F000324A3121C68FEAFF0900320E0FD12288F
:101B8F00FB12342F900322E475F0011208519003D9
:101B9F001FE004F0E0C3940D40BA90031CE004F082
:101BAF0090031EE004F0021B3212378C121C8C7A49
:061BBF002E79AC122EEDA0
:101BC5002290031CE075F00BA424C4F9741035F0C1
:071BD500FA7BFF1226BE227D
:0B1EEE00900318EFF0A3EDF0A3EBF061
:101EF900E490031FF0A3F090031F121D0840030292
:101F09001FAD9010CB75F00BEF121C3590031CF030
:101F19006422607C90031F121C447F011226BE902C
:101F2900031CE0FF900318E0FDA3E0FBA3E090038E
:101F390029F090031BE090032AF0123191E49003F9
:101F49001EF01230DAEF60379003C0E06430702F72
:101F590090031C121CA06F702690031FE0FEA3E0E3
:101F6900FF121C457F041226BE1230DAEF60FA9088
:101F790003C0E0B42FF390031C121CA0B507EA7F3D
:101F89000112347590031EE004F0E0C3940540B2D9
:101F9900900320E004F06003021F0090031FE00497
:101FA900F0021F007BFF7A1179C17F041226BE90CF
:101FB900031AE0FB900318E0FED39B4040EE121D8C
:101FC90016EB1490031EF0900319121CCCD3121DAA
:101FD9005C5070121BDCE490031DF0121C57122098
:101FE9005640F812342F900320E004F07006900355
:101FF9001FE004F090031EE004F0021FD0900319C3
:10200900E0121D1690031BE01490031EF0900318B4
:10201900121CCCC3121D5C402A121BDCE490031D68
:10202900F0121C5712205640F812342F900320E06A
:1020390024FFF090031FE034FFF090031EE014F03A
:0D204900022016121C8C7A2E79AC022EEDAE
:1020560085F082F583E493FD1228FB90031DE004CE
:06206600F0E0C3940D221E
:1037C500203025252000253264252520003530258B
:0237D5002500CD
:102BEC009003BDE0FEA3E0FFD390031DE09F900394
:102BFC001CE09E22EFFD900341E0FB3395E0FAC30D
:102C0C00EB9D7480F86A98229003B97402F09003DB
:102C1C00BD747FF0A374FFF02274FF90033FF0C2E9
:102C2C00032290031CE0FCA3E0FFECFD22E0F5C1C5
:072C3C00A3E024FF92AF2288
:1015C200E490032EF0A3F090031874A0F0122C14F0
:1015D200A2AFE43390031AF0C2AF900319E5C1F051
:1015E20090031BE5CBF043C15E75CBEB900318E093
:1015F200FB7423122C27E4FDFF12248D900318E0C4
:10160200FB90033F7421F0C2037F0112172B743247
:10161200F0C2037F0212172B7430F0C2037F031251
:1016220017397430F0C2037F041217397445F0C2BF
:10163200037F051217867450F0C2037F06121786C5
:101642007453F0C203E4FD7F0712248D90032EE44D
:10165200F0A37408F01217A57437F0A374C5F0E470
:10166200A312179412310A90031CE4F0A37408F039
:10167200122BEC504290032FE004F0700690032EE0
:10168200E004F090032EE064027004A3E0648F7023
:101692000D121762900340EE12174712310A122CF4
:1016A2002E900318E0FB122C251217B4700690033B
:1016B2001CE004F00216721217A57437F0A374D25C
:1016C20012179412310AE490032EF0A3F090031C37
:1016D200F0A3F0122BEC504490032FE004F07006BC
:1016E20090032EE004F090032EE064027004A3E065
:1016F200648F7012121762EF2432FFE43E900340AF
:1017020012174712310A122C2E122C257BA2121705
:10171200B4700690031CE004F00216D590031BE09F
:08172200F5CB900319122C39DC
:10172A0022E4FD12248D900318E0FB90033F22E48B
:10173A00FD12248D900318E0FB90033F22F0A3EFE3
:10174A00F07B017A03791E120B11E490032EF0A3A9
:10175A00F07B017A03791E22FD7F011238C89003BB
:10176A003D74FFF0A37437F0A374CBF090031CE030
:10177A00FEA3E0FF7C027D8F1207FC22E4FD122407
:10178A008D900318E0FB90033F22F07B017A0379E6
:10179A001E120B117B017A03791E22E4FD7F0112CE
:1017AA0038C890033D74FFF0A32212248D90031DC4
:0417BA00E004F02235
:10256F00C202A2AFE433900339F0C2AF900338E553
:10257F00C1F043C15EE490032FF090032FE0FFC33F
:10258F0094085045E490033FF0D2037BA0FD122442
:10259F008D90032FE02430F582E43403F583EFF0C0
:1025AF00E490033AF0A3F090033BE004F070069040
:1025BF00033AE004F090033AE0B413EBA3E0B488DD
:0125CF00E625
:1025D00090032FE004F080B1900330E06423702674
:1025E000A3E064217020A3E06432701AA3E0B43049
:1025F00015A3E0B43010A3E0B4450BA3E0B450063B
:10260000A3E064536004C2028002D2029003381235
:0B2610002C39300205122C14D322C319
:01261B00229C
:08248D0090033CEFF0A3EDF019
:10249500A2039207C2092014FDD214900340EBF069
:1024A500C204D205D2087F01C2C4C20AD2C530C057
:1024B500FDE5C054F02480607624C0601B24E060F4
:1024C50003022554900340E0F5C2A204E43342C25E
:1024D500C2C5E4A3F002255630C149300A07D2C56A
:1024E500C20A02255630050CC205D20690033DE00E
:1024F500F5C2805D300611C20690033CE0F5C2309E
:10250500074FD20AD2048049200446122C00500EEF
:1025150090033FE0F5C2900341E004F08033D2C45C
:10252500C214802D300804D2C58026D2098022121B
:102535002C00500CA3E5C2F0900341E004F0D2C199
:10254500900341E0B5070AC214C2C1D2C48002D2C9
:102555000930090853C0BF43C040C214C2C030147B
:09256500030224B3900342E0FFDD
:01256E00224A
:02362200C10CD9
:1034DA0075120375137D22850E0A850F0B2214F5CA
:1034EA00828C83E0F5C2EF650B22750A03750B7DAA
:0134FA0022AF
:0B392400D2CB438E2075CBAED2CA225E
:1037FB0075C102E4F5C2F5C053C17F43C1800239E4
:01380B002498
:1033C2007E037F698E0C8F0D8E108F118E088F09F0
:1033D2007E037F7D8E0E8F0F8E128F138E0A8F0BC0
:0533E200C20B0237FBE5
:10300D000511E511AA107002051014F5828A83EFDF
:10301D00F0AF050511E511AC107002051014F58225
:10302D008C83EFF0747DB5110B7403B5100675101C
:05303D0003751169227A
:0C38D400E5C120E5FBC20BC2C4D2C52236
:10198F00200B3FD20B0513E513AC12700205121496
:10199F00F5828C8374FFF07C037D91EDB51307EC1A
:1019AF00B512031234DA0513E513AA1270020512E9
:1019BF0014F5828A83E4F0EDB51307ECB512031228
:1019CF0034DA0513E513AC127002051214F5828C8C
:1019DF0083E4F07C037D91EDB51307ECB512031290
:1019EF0034DA0513E513AA127002051214F5828A70
:1019FF0083EFF0EDB51307ECB512031234DA7F0164
:011A0F0022B4
:10355800E509B50D08E508B50C037F0022850D8245
:0D356800850C83E0B507037F01227F002260
:10321100050DE50D7002050C050DE50DAE0C7002F6
:10322100050C14F5828E83E0FF747DB50D0B7403DC
:09323100B50C06750C03750D695E
:01323A002271
:061A27007FFF123558227A
:06395400E4FF12355822C9
:031A1800021D6646
:101D6600C0E0C083C082C0D075D000C000C002C031
:101D760004C005C006C007E5C054FE1209C91EB856
:101D8600081EB80A1ECE0C1ECE0E1E9A101E9A12E1
:101D96001EAD141EAD161E921C1E921E1E8E241EF5
:101DA6008E261E56281E562A1E622C1E622E1DF5D3
:101DB600C01DFFC21DC4E01DC4E200001ED7C2C57F
:101DC600050BE50B7002050A7E037F91B50707EE4A
:101DD600B50A031234F4050BE50BAC0A7002050ACA
:101DE6001234E87003EE650A6003021ED7805B12A8
:101DF60034E1D2C4D2C5021ED7E50BB51312E50AEB
:101E0600B5120D85120E85130FC2C5D2C4021ED798
:101E1600850B82850A83E0B4FF03021ED3050BE51A
:101E26000B7002050A7E037F91B50707EEB50A031C
:101E36001234F4050BE50BAC0A7002050A1234E8FD
:101E46007003EE650A6003021ED71234F4021ED731
:101E5600E5C26023E5C26421601D80111234E1C22F
:101E6600C5D20CE5C26010E5C26421600AC2C4C2D4
:101E7600C5C2C1C20D805AADC27FFF12300DC2C4A9
:101E8600C2C5D2C1D20D8049D2C58045850A0E850C
:101E96000B0F803D851008851109C2C4C2C1300CE4
:101EA60030D2C5C20C802A1234E1C2C4C2C1D2C526
:101EB600801FC2C4C2C5200D04C2C18014ADC2E4D5
:101EC600FF12300DD2C180091234E1C2C1C2C4D2A0
:101ED600C5C2C0D007D006D005D004D002D000D0ED
:081EE600D0D082D083D0E0329D
:1013420025326420002E3500312E3000312E35003A
:10135200322E30004D6F7270682054696D653A25E7
:10136200737300006F6666006F6E0052656D6F7476
:10137200650042617365204368616E6E656C3A2058
:1013820025326400456E61626C6564004469736174
:10139200626C65640053746174757300466F726D9C
:1013A200617474696E67204361726400202020209A
:1013B2002020446F6E6520202020200020004469F8
:1013C200737020436F6E74726173743A20256400E7
:1013D200466F726D61742043617264004D6F647573
:1013E2006C65202573004669726D777265205665BB
:1013F2007273202564002020436F7079696E672024
:1014020066726F6D2000202020436F7079696E67CD
:1014120020746F20200020202020506F6C6C696E99
:1014220067202020200020202020436F7079696EE1
:1014320067202020200020202045786368616E67A5
:10144200696E6720202020002020204D6F64756C7B
:1014520065202573202020002532642D2532643A30
:101462002532642D25326400436F707920457863FC
:1014720068616E676500436F707920437264203E35
:101482002031362D333000436F70792031362D33C1
:1014920030203E2043726400204142434445464787
:1014A20048494A4B4C4D4E4F505152535455565742
:1014B20058595A6162636465666768696A6B6C6DE4
:1014C2006E6F707172737475767778797A303132A3
:1014D200333435363738397E21402324255E262A97
:1014E20028292D2B3D7C01028D339C01029C380C56
:1014F200010299351B01029536D00102EA35AC0191
:1015020002FE36E6010303373B0102D236E6010250
:10151200D5373B000000000001028D35FA01029C24
:101522002F680102FE394B01030338A20102992EF2
:10153200650102D239680102D53968000000000055
:1015420001028D2B2A01029C2F68010299385B014E
:1015520002FE36A2010303367300000000000102FE
:101562008D261C01029C38E00102FE36A201030313
:1015720036730000000000FF1347FF134AFF134EAB
:10158200FF1352FF1366FF136A0007FF38AF010F04
:10159200FF3778000FFF36B90100FF33760001FFF5
:1015A20027570004FF27EE0007FF2A530100FF37E9
:1015B200E90105FF37D70000FF38860100FF3894A4
:06362400C10F4102D800B5
:1023A90090033D7401F0A37402F074EDA3F07B0176
:1023B9007A0279D922A3F090033D74FFF0A3229009
:1023C9000299F0A3EAF0A3E9F022900292E0FBA3BC
:1023D900E0FAA3E0F922A3F07B017A0279ED22D297
:1023E9000F900289A3E0FF900308A3E0FD90030684
:1023F900A3E0FB900301E0F8A3E022E0F9A3E0FAEF
:10240900A3E022900289E0FEA3E0FF22A3F090025C
:102419009C74FFF0A32290028D74FFF0A322900216
:10242900927401F0A32275F005A424A1F582E43485
:1024390002F5832275F005A4249FF582E43402F5A0
:10244900832275F005A424A0F582E43402F58322E1
:102459007B01AD0790031CF0229EFED3EF940EEE94
:102469006480948022E02401FEE433900340F0224A
:10247900A3F09002FE74FFF0A322A3F0900303746B
:04248900FFF0A3229B
:0A392F00E490028CF090028BF0226D
:06395A00E4900298F02247
:1029750090033AEEF0A3EFF0AF051DEF6061900311
:102985003AE0FEA3E0F5828E83A3A3E493FB7401F2
:1029950093FA740293F9900298E0FF12242FEB1238
:1029A50023CB90033AE0FAA3E0FBF5828A83E49314
:1029B500FEEF12243DEEF08B828A83740193FF9023
:1029C5000298E012244BEFF0900298E004F0900397
:1029D5003BE02405F090033AE03400F002297D2223
:103350001223D312079DFE12243DE0FFEE12244BF0
:10336000E0FD1238C81223D312079D12242F122415
:0633700004C91223C8226B
:1036A2001223D312079D7007900298E01207D812D6
:0736B20023D374FF0207B6E9
:103673001223D374011207B612079DFF900298E03C
:08368300B50704E41207D82288
:01396600223E
:1032DC007BFF7A3979669002EAEB1223CB90029548
:1032EC00EB1223CB9002FEEB1223CB900303EB12D9
:0732FC0023CBEB1223C822D3
:102E1D00900318EB1223CB1232DC9003181223D639
:102E2D0012095AEA494B602F9003181223D69000CD
:102E3D000312087DAAF0F97BFFC003C002C0019008
:102E4D0003181223D612095A12097A900319E47540
:082E5D00F00512085180C322A8
:0C2AC100900318EFF0A3EBF0A3EAF0E99B
:102ACD001223BE7413F0A37442F0ED2401FEE4331F
:102ADD00A3F0A3CEF07B017A03791C120B119003A6
:102AED0018E0FFE4FD1238C87B017A03791C12311E
:102AFD000AE4FD900319E0FBA3E475F001120867E9
:102B0D00A9F0FA12079D90149A93FF1238780DEDE3
:0D2B1D00B40DE0900318E0FF7D010238C800
:01396700223D
:10351B0090039FE02FF0E0FFB41E04E4F0800AEF6D
:0F352B00B4FF0690039F741DF012378C023967AE
:10373B0090039FE004F0E0B41E02E4F012378C1209
:05374B0039670236D0D1
:1036E60090039FE014F0E0B4FF03741DF012378CD2
:0636F6001239670236D014
:102E65009002D1E0FE7C0024A4F9EC3403FA7B0146
:102E7500EE601A12079D70159002D1E024A3F58229
:102E8500E43403F583E060051207D88004EF1207E8
:102E9500B612079DFFB44E04744D8005EFB4FF04D0
:062EA500E41207D8D2126E
:012EAB002204
:09394B009002D1E0600214F022A8
:0D38A2009002D1E0C3940C5003E004F0222A
:10357500ED1207B612079DFFB4FF03E4800A90031E
:0C3585001CE0FEB50705EE141207D8226A
:0F385B007A0379B17404122459123575D21122EF
:0D38AF00EFB40104D20E8002C20ED210222E
:1036B9007A0379B374081224591235759003B3E06B
:0736C900FF12353AD2112275
:103778007B017A0379B4AD0790031C7410F01235FD
:0437880075D21122C3
:01396800223C
:102F680012379F12241F7422F0A374BEF0C21012ED
:102F780024177437F0A374B2F090029974FFF0A389
:102F88007438F074AF1224797436F074A212248362
:082F98007436F0A37473F022FB
:1037B20012241F742BF0748D1224157430F0A3742C
:0337C20076F0227C
:10380C007BFF7A15791A122E1DE49002D1F0C212A8
:01381C002289
:0C38E00012379F7BFF7A1479E8022E1D3E
:102B2A007D027FF31238F81223C07413F0A374568F
:102B3A00F09003B1E075F003A42479F582E434152A
:102B4A00F583E493F9740193FA740293900340C9EC
:102B5A001223CB7B017A037918120B1190033D746F
:102B6A00FFF0A37413F0A37465F07B017A0379185C
:102B7A001231387E037F1812368BEF24FEFDE4FFF4
:032B8A000238C846
:1022BE007D027FF31238F81223C07413F0746D127E
:1022CE0023B5120B111223C07413F0A37474F09083
:1022DE0003B412246ECE1223DF120B111223A91295
:1022EE0031387D07E4FF1238C820100302238730EF
:0922FE000E7CE4900318F0A3F03B
:1023070090031A12091D00000000E47F407E9CFD27
:10231700FC90031AE0F8A3122404FBC31208B5507B
:102327002790031AE0FCA3E0FDA3E0FEA3E0FFE48F
:10233700FAF9F8EF2401FFEA3EFEE93DFDE83CFC2F
:0823470090031A12091180C273
:10234F00123919123903900319E004F07006900343
:10235F0018E004F0C3900319E09403900318E064AD
:10236F0080948040937BFF7A137986801112390E07
:10237F007BFF7A13798E80067BFF7A137997123160
:10238F000A12395A7E157F8B7D0212297512242766
:0A239F007402F0A3748BF0023350B7
:103452001223C07413F0A3749E1223B6120B11121E
:1034620023C07413F074651223DF120B111223A907
:03347200023138EC
:10337600EFB40121D20F1234521215C290033274E7
:10338600FFF0A37413F0A374BEF07BFF7A1379AE3B
:06339600122EEDC20F2211
:102B8D001223C07413F0A374C0F09003B312246E1B
:102B9D00A3CEF07B017A037918120B111223C074A6
:102BAD0013F0A374D2F07B017A037929120B1190E3
:102BBD00033D7401F0A37403F0A37429F07B017A33
:102BCD0003791812313812395A7E157F957D02120C
:0F2BDD0029751224277402F0A3748CF002335070
:10382D0090039FE0FD7B017A0379A47F01022AC1F9
:1035FA007D047FF51238F812396012382D9002D105
:09360A00E02403FD7F010238C831
:10339C007D087FF91238F8123960900391E075F0CE
:1033AC000DA42479F9743A35F0FA7BFFE0FDE4FFC3
:0633BC00122AC102382DA7
:08347500AB07AF031BEF601A67
:10347D0090033512091D0000445C90033574FF1252
:0A348D0008DEEC4D4E4F60E280F0C7
:013497002212
:102C4300900313EB1223CBA3ECF0ED1223BE74130A
:102C5300F0A374DEF0900313122404900340C9F030
:102C6300A3EAF0A3E91223B6120B111223C07413C3
:102C7300F0A374E8F0900316E0FFA3E0900340CFC5
:102C8300F0A3EF1223E0120B111223A91231387FA4
:072C9300321234750238EC27
:0C38EC0090028D1223D81209EF02316502
:10275700EFB40126900289E07004A3E0641E700ABA
:10276700900289F0A3741EF0803B90028AE004F087
:102777007033900289E004F0802BD390028AE094B2
:1027870001900289E064809480401A900301E07010
:1027970004A3E0641E600E90028AE024FFF090021A
:1027A70089E034FFF012240CC3900309E09FEE6424
:1027B70080F8900308E06480985005EEF0A3EFF0EE
:1027C700C3900309E09FFF900308E01224624014BE
:1027D70090028AE0240EFE900289E03400900308FC
:0727E700F0A3CEF00238EC74
:1027EE00EFB40132900308E07004A3E0641E700A97
:1027FE00900308F0A3741EF08051900301E0700462
:10280E00A3E0641E6045900309E004F0703D900360
:10281E0008E004F0803512240C900308E0FCA3E0DD
:10282E00FDB5070EECB5060A900308EEF0A3EFF027
:10283E008019D3ED9401EC64809480400E900309CE
:10284E00E024FFF0900308E034FFF012240C900314
:10285E0008E0FCA3E0FDC39FFFEC122462400EEDE6
:10286E0024F2FEEC34FF900289F0A3CEF00238EC95
:102A5300900289A3E0FE900308A3E0C39EFEEFB4B7
:102A6300013C900306E0FCA3E0FD641E4C700A9059
:102A73000306F0A3741EF08042AF067E00ED2FFF25
:102A8300EE3CFEC3EF941EEE64809480502D9003C1
:102A930007E004F07025900306E004F0801DD39056
:102AA3000307E09401900306E064809480400CA344
:0E2AB300E024FFF0900306E034FFF00238EC60
:1037D700EF6401700C1223E890031BF0121A30C239
:0237E7000F22AF
:102EED0090032FEB1223CB90032F12240490033D5C
:102EFD00C9F0A3EAF0A3E91223B6120B1190033225
:102F0D0012240490033DC91223CB1223E1120B119D
:0E2F1D001223A91231387F1E1234750238ECCF
:1026BE00900330EB1223CB90032FEFF0BF020F12DB
:1026CE0023C07413F0A374F81223B6120B119003E7
:1026DE002FE0B4030F1223C07414F0A37408122356
:1026EE00B6120B1190032FE0B4010F1223C0741415
:1026FE00F0A374181223B6120B1190032FE0B4043A
:10270E000F1223C07414F0A374281223B6120B11E7
:10271E0090032FE0B4050F1223C07414F0A3743885
:10272E001223B6120B111223C07414F0A3744AF0C4
:10273E00900330122404900340C91223CB1223E1DC
:09274E00120B111223A90231380B
:1037E900EF6401700C1223E890031BF0121EEEC265
:0237F9000F229D
:0E388600EFB40109D20FD200120E11C20F22B0
:0E389400EFB40109D20FC200120E11C20F22B2
:1030760012241F7426F0741C1224157434F0A374E1
:103086000BF0900289E4F0A304F0900308E4F0A3A7
:1030960004F0900306E4F0A304F0900301E4F0A327
:0330A60004F02211
:10261C0012240C900308E0FAA3E0FBC39FFFEA9E90
:10262C00FE900306E0FCA3E0FD2FFFEC3E900301BF
:10263C00F0A3EFF012240CC3EB9FEE6480F8EA6475
:10264C0080985007E4900301F0A3F01223C0741497
:10265C00F0A3745AF0A3EEF0A3EFF0900308E0FFA0
:10266C00A3E0900342CFF0A3EFF0A3ECF0A3EDF0C6
:10267C00900301E0FFA3E0900346CFF0A3EF1223F9
:10268C00B6120B111223C07414F0A3746A1223E057
:10269C00120B111223A912313812395A7E157F9F51
:1026AC007D051229751224277402F0A37490F00290
:0226BC00335099
:10340B0012241F742FF0A3742B1224167438F0742B
:10341B00E01224797436F074A21224837436F0A36C
:04342B007473F022A4
:102F2B001223C07414F0A374781223B6120B11126F
:102F3B0023C07414F0A374891223E0120B11122313
:102F4B00A912313812395A7E157FB87D02122975B4
:0D2F5B001224277402F0A37491F002335089
:03000000020600F5
:03000300021A03DB
:03000B00021A06D0
:03001300021A09C5
:03001B00021A0CBA
:03002300021A0FAF
:03002B00021A12A4
:03003300021A1599
:03003B00021A188E
:03004300021A1B83
:03004B00021A1E78
:03005300021A216D
:03005B00021A2462
:03006300021A2757
:03006B00021A2A4C
:03007300021A2D41
:10060000E4F5D9E5EF7480F5FF7402F5EF787FE447
:10061000F6D8FD9000007F007E04E4F0A3DFFCDE4E
:07062000FA75812902066250
:100627000217BEE493A3F8E493A34003F68001F214
:1006370008DFF48029E493A3F85407240CC8C333D4
:10064700C4540F4420C8834004F456800146F6DFA3
:10065700E4800B0102040810204080903613E47EEA
:10066700019360BCA3FF543F30E509541FFEE49398
:10067700A360010ECF54C025E060A840B8E493A35F
:10068700FAE493A3F8E493A3C8C582C8CAC583CA8A
:10069700F0A3C8C582C8CAC583CADFE9DEE780BE42
:01362A00009F
:1006A700E709F608DFFA8046E709F208DFFA803E35
:1006B70088828C83E709F0A3DFFA8032E309F60822
:1006C700DFFA8078E309F208DFFA807088828C838A
:1006D700E309F0A3DFFA806489828A83E0A3F6083E
:1006E700DFFA805889828A83E0A3F208DFFA804C18
:1006F70080D280FA80C680D4806980F280338010EF
:1007070080A680EA809A80A880DA80E280CA803357
:1007170089828A83ECFAE493A3C8C582C8CCC583CF
:10072700CCF0A3C8C582C8CCC583CCDFE9DEE7809F
:100737000D89828A83E493A3F608DFF9ECFAA9F01E
:10074700EDFB2289828A83ECFAE0A3C8C582C8CC74
:10075700C583CCF0A3C8C582C8CCC583CCDFEADE8D
:10076700E880DB89828A83E493A3F208DFF980CCEF
:1007770088F0EF60010E4E60C388F0ED2402B404E8
:100787000050B9F582EB2402B4040050AF2323458F
:0607970082239006F773B7
:10079D00BB010689828A83E0225002E722BBFE025A
:0907AD00E32289828A83E493228D
:1007B600BB010989828A83F8E028F022500327F7D3
:1007C60022BBFE05F8E328F3228A838982F8E493A4
:0207D6002822D7
:1007D800BB010689828A83F0225002F722BBFE0100
:0207E800F322FA
:1007EA00EF8DF0A4A8F0CF8CF0A428CE8DF0A42E23
:0207FA00FE22DD
:1007FC00BC000BBE0029EF8DF084FFADF022E4CCE1
:10080C00F875F008EF2FFFEE33FEEC33FCEE9DECA9
:10081C00984005FCEE9DFE0FD5F0E9E4CEFD22EDEF
:10082C00F8F5F0EE8420D21CFEADF075F008EF2F39
:10083C00FFED33FD4007985006D5F0F222C398FD2A
:05084C000FD5F0EA22C7
:10085100C5F0F8A3E028F0C5F0F8E5821582700232
:060861001583E038F022CF
:10086700A3F8E0C5F025F0F0E58215827002158344
:06087700E0C838F0E822A1
:10087D00BB0110E58229F582E5833AF583E0F5F0B9
:10088D00A3E0225009E92582F886F008E622BBFE96
:10089D000AE92582F8E2F5F008E222E5832AF583DC
:0808AD00E993F5F0A3E99322A1
:1008B500EB9FF5F0EA9E42F0E99D42F0EC6480C8BA
:0608C50064809845F0225A
:1008CB00EB9FF5F0EA9E42F0E99D42F0E89C45F083
:0108DB0022FA
:1008DC007401FF3395E0FEFDFCA3A3A3E0CF2FF042
:1008EC00E582158270021583E0CE3EF0E58215821A
:1008FC0070021583E0CD3DF0E58215827002158300
:05090C00E0CC3CF022EC
:0C091100ECF0A3EDF0A3EEF0A3EFF02259
:10091D00A8828583F0D083D0821209341209341253
:10092D000934120934E473E493A3C583C5F0C58378
:10093D00C8C582C8F0A3C583C5F0C583C8C582C824
:01094D002287
:0C094E00A42582F582E5F03583F58322B4
:10095A00BB010789828A83020A655005E9F8020AFF
:10096A0053BBFE05E9F8020A8E89828A83020AA02D
:10097A00BB011A89828A83D0F0D0E0F8D0E0F9D09E
:10098A00E0FAD0E0FBE8C0E0C0F0020A855016E9C0
:10099A00F8D083D082D0E0F9D0E0FAD0E0FBC08270
:1009AA00C083020A5CBBFE16E9F8D083D082D0E08D
:0F09BA00F9D0E0FAD0E0FBC082C083020A972296
:1009C900D083D082F8E4937012740193700DA3A3BD
:1009D90093F8740193F5828883E4737402936860D1
:0609E900EFA3A3A380DFD1
:0609EF008A838982E47393
:1009F500E5292582F582E5283583F583B528048523
:100A050082292210AF06858229F52822858229F5BB
:040A150028D2AF2212
:0D0A1900E5292582F582E5283583F5832245
:100AAC00E523243DF582E43403F583E0052322900D
:100ABC00033A30090390033DE475F001120A6E020B
:100ACC00079D2002E97F2ED2028018EF540F24904C
:100ADC00D43440D4FF30060BEF24BFB41A005003BB
:100AEC002461FFE524600215240527E52770020523
:100AFC002630090E90033AE475F001120A6EEF02EB
:100B0C0007D80233037403D2098003E4C209F52326
:100B1C0090033A120A85E4F524F526F527E52460BE
:100B2C00077F20120AEF80F57525FFC203C202C2AF
:100B3C0004C205C207C208C20A120ABBFF700D30FC
:100B4C0009057F00120B00AF27AE2622B4255FC229
:100B5C00D5C206120ABBFF24D0B40A00501A75F095
:100B6C000A782430D50508B6FF0106C6A426F6205F
:100B7C00D5047002D20580D924CFB41A00EF5004EA
:100B8C00C2E5D206020D01D20380C6D20280C0D2C9
:100B9C000480BCD2D580BAD20780B47F20120AEF71
:100BAC002004077401B5240040F1120AACFF120AAC
:100BBC00EF020B29D20AD2088095120AACFB120A5A
:100BCC00ACFA120AACF94A4B700679D27A0D7BFF5B
:100BDC0020042EE524602A7E008E82758300120A82
:100BEC002660060EEE652570F0C2D5EBC0E0EAC0BB
:100BFC00E0E9C0E0EE120D48D0E0F9D0E0FAD0E028
:100C0C00FB12079DFF60AAEBC0E0EAC0E0E9C0E080
:100C1C00120AEFD0E02401F9D0E03400FAD0E0FB66
:100C2C00E5250460DCD525D980877BFF7A0D7944D6
:100C3C00D204809C791080027908C208C20A80080C
:100C4C00D2D5790A8004790AC2D5E525047002F55B
:100C5C0025E4FAFDFEFF120AACFC7B0820031312FC
:100C6C000AACFD7B1030020A120AACFE120AACFF71
:100C7C007B20EC3382D592D55013C3E43002069F0F
:100C8C00FFE49EFEE42003039DFDE49CFCE4CBF812
:100C9C00C203EC700CCFCECDCCE824F8F870F38006
:100CAC0017C3EF33FFEE33FEED33FDEC33FCEB33C8
:100CBC00FB994002FB0FD8E9EB300305F8D0E0C4F8
:100CCC0048B203C0E00AEC4D4E4F78207B0070C256
:100CDC00EAB5250040BCC0E0120D4AD0F0D0E020AF
:100CEC000304C4C0E0C4B203C0F0120AD8D0F0D5DB
:100CFC00F0EB020B291209C90BC6530C40580B9789
:100D0C004C0B93420C444F0C4C440C4C490BAC43D5
:080D1C000C52550C36460C3652
:100D2400450C36470DF2500B9B2D0B9F2E0BC22BFF
:100D34000BA3230BC0200DDB2A0B5B4800000BBA6E
:100D44003F3F3F00790AA2D5200514300709B910A6
:100D5400020404B9080104A2D520080250010420A9
:100D640004689204B524005034C0E07F2030051993
:100D74007F30A20472087207500F120DA1C204C280
:100D840008C207C20A7F30800F300703E9C0E012AF
:100D94000AEF300703D0E0F9D0E0B524CC300717D0
:100DA4007F30B9100C120AEF7F583006077F788025
:100DB40003B90803120AEF3004057F2D020AEF7FFE
:100DC40020200AF87F2B2008F322920480CF286E7B
:100DD400756C6C2900D203120AAC3003F8C2037894
:100DE4002430D50108F6020B5B2D50434958120AF2
:100DF400AC2403B405004001E4900DED93120AE025
:0D0E0400743A120AE0D205752404020C4075
:100A2600BB010CE58229F582E5833AF583E0225085
:100A360006E92582F8E622BBFE06E92582F8E222CF
:0D0A4600E58229F582E5833AF583E49322E9
:090A5300E6FB08E6FA08E6F922C8
:090A5C00EBF608EAF608E9F622BF
:090A6500E0FBA3E0FAA3E0F92292
:100A6E00F8E0FBA3A3E0F925F0F0E5821582700211
:070A7E001583E0FA38F022B5
:090A8500EBF0A3EAF0A3E9F02272
:090A8E00E2FB08E2FA08E2F92299
:090A9700EBF208EAF208E9F22290
:0C0AA000E493FB740193FA740293F922B2
:10330300EFB40A07740D12330E740A309811A8999A
:10331300B8130CC2983098FDA899C298B811F6302A
:0733230099FDC299F5992202
:00000001FF
